:100000000C94CA000C94E7000C94E7000C94E700F1
:100010000C94E7000C94D8020C94E7000C94E700D1
:100020000C94E7000C94E7000C94E7000C94E700B4
:100030000C9483170C94E7000C94E7000C94E700F1
:100040000C94B1020C94E7000C94E9000C94E700C6
:100050000C94E7000C94E7000C94E7000C94E70084
:100060000C94E7000C94E7000C94E7000C94E70074
:100070000C94E7000C94E7000C94E7000C94E70064
:100080000C94E7000C94E7000C94E7005D0D5F0D05
:10009000610D630D650D670D690D6B0D6D0D6F0DB8
:1000A000710D730D750D770D790D7B0D7D0D7F0D28
:1000B000810DC30DC30DC30DC30DC30DC30D830D42
:1000C000850D870D890D8B0D8D0D8F0D910D950D66
:1000D000990D9F0DA30DA70DAB0DAF0DB50DB70D70
:1000E000B90DBD0D0D0E0F0E110E130E150E170EC0
:1000F000190E1B0E1D0E1F0E210E230E250E270E90
:10010000290E2B0E2D0E2F0E310E730E730E730E45
:10011000730E730E730E330E350E370E390E3B0E03
:100120003D0E3F0E410E450E490E4F0E530E570E1B
:100130005B0E5F0E650E670E690E6D0EAF0EB50E8F
:10014000BB0EC10EC70ECD0ED30ED90EDF0EE50EBF
:10015000EB0EF10EF70EFD0E030F090F0F0F150F2B
:100160001B0FAC0EAC0EAC0EAC0EAC0EAC0E210FD9
:10017000270F2D0F330F390F3F0F450F4B0F550F23
:10018000610F6B0F750F7F0F890F930F9D0FA30FDB
:10019000A90FAF0F11241FBECFEFD0E1DEBFCDBF3F
:1001A00011E0A0E0B1E0E4E6F3E300E00BBF02C041
:1001B00007900D92A435B107D9F714E0A4E5B1E09A
:1001C00001C01D92A93BB107E1F70C94F3000C9418
:1001D00000001F920F920FB60F9211240F900FBEC6
:1001E0000F901F901895CCEFD0E1DEBFCDBF8FEF01
:1001F00087BB88BBC7980E94270781E897E10E94C8
:10020000720785E69CE00E94770781E090E00E94FB
:100210007C07DE011196EBE4F1E083E001900D92A2
:100220008150E1F7CE0101960E94710B80E091E0D0
:100230000E940D0C81E191E00E94050C82E491E0A6
:100240000E94FD0B0E94470B4C0164E670E00E9487
:100250008A0760E070E0C4010E94B30A3C0140E0FC
:1002600050E0BC01C4010E94AB0720ECA22E21E0AB
:10027000B22ECC24DD2490E4E92EF12C02E021E022
:1002800030E041E050E0B301C4010E94480A87E435
:10029000A82E82E0B82E21E030E041E050E0B3012A
:1002A000C4010E94800A0E94C1061092E1011092CE
:1002B000E0011092E3011092E2010E943B0C8FEFEB
:1002C00084BB8AEA85BB0E94FC0285ED85BB0E9447
:1002D000FC0280E885BBFFCF0F931F93CF93DF9382
:1002E000EC0181349105B0F08091EC019091ED0129
:1002F000892B81F41092E9011092E801D093EB016F
:10030000C093EA0181E090E09093ED018093EC01CD
:10031000C0E4D0E068E08BE20E94100700E010E04B
:100320000EC0E091E801F091E901E00FF11FEE5CF1
:10033000FC4F608189E20E9410070F5F1F4F0C176E
:100340001D0779F78091E0019091E101019749F44F
:1003500067E08BE20E9410071092E1011092E00129
:100360000AC063E08BE20E94100781E090E0909366
:10037000E1018093E001DF91CF911F910F910895EA
:100380008091EC019091ED01019771F52091E801C8
:100390003091E9018091EA019091EB01281739072A
:1003A00018F52091EA013091EB018091E8019091DC
:1003B000E901281B390B8091E8019091E901805CEB
:1003C0009F4F9093E9018093E801213431052CF08F
:1003D00080E490E00E946C010895C9010E946C01C4
:1003E0001092ED011092EC010895FC011092E901C8
:1003F0001092E8011092ED011092EC010000C79AF2
:100400002081822F82958F7099278230910511F17A
:10041000833091052CF4009761F0019759F516C0CF
:1004200084309105F9F084309105C4F0059711F5F9
:100430001DC0263039F48281813039F5CF010E9408
:10044000501723C0CF010E94B50C1FC0CF010E94DE
:10045000DD111BC0CF010E94FB1217C0CF010E940B
:100460003B1413C0CF010E946A150FC0CF010E9438
:100470002E180BC02093320383E080933303109235
:10048000340383E090E00E946C01C7980895CF93F5
:10049000DF93EC018091E2019091E301019751F526
:1004A00020E030E0E091E401F091E501E20FF31F7C
:1004B000DE01A20FB31F8C91EE50FE4F80832F5FA1
:1004C0003F4F2034310571F78091E4019091E501AF
:1004D000805C9F4F9093E5018093E4012091E401BB
:1004E0003091E5018091E6019091E70128173907E5
:1004F000A8F11FC01092E5011092E40120E030E065
:10050000E091E401F091E501E20FF31FDE01A20F9B
:10051000B31F8C91EE50FE4F80832F5F3F4F2034EE
:10052000310571F73093E5012093E401A981A034EE
:1005300048F41092E3011092E20182EF91E00E94F0
:10054000F5010CC081E090E09093E3018093E2011B
:100550008A2F99279093E7018093E601DF91CF914D
:1005600008951F920F920FB60F9211242F933F936D
:100570004F935F936F937F938F939F93AF93BF93AB
:10058000EF93FF930E94860C80915D0182BFFF91E3
:10059000EF91BF91AF919F918F917F916F915F91FB
:1005A0004F913F912F910F900FBE0F901F90189574
:1005B0001F920F920FB60F9211242F933F934F93D8
:1005C0005F936F937F938F939F93AF93BF93EF93BB
:1005D000FF930E94150CFF91EF91BF91AF919F91F6
:1005E0008F917F916F915F914F913F912F910F90DC
:1005F0000FBE0F901F90189520E080E49CE90197B2
:10060000F1F72F5F2931C9F70895FF920F931F93D8
:10061000162F042FF22E9C01442737FD4095542FAE
:1006200060E472E48FE090E00E9461192150304054
:10063000163061F0173019F0153019F404C0E1E0FC
:1006400003C0E1E004C0E0E070E002C0E0E071E07F
:10065000053439F00F3419F451E041E004C050E0A2
:1006600001C051E040E082E0F81611F462E001C000
:1006700060E0832F992787FD9A958093900029B990
:1006800088E18AB9770FEE0FEE0FE72B5295550FE1
:10069000507E5E2B4295407F452B660F660F660F9E
:1006A000642B609395001F910F91FF900895109215
:1006B000900089E189B988E18AB986E08093950044
:1006C000089508955D9BFECF8CB908955F9BFECF82
:1006D0008CB1992708958A3310F4805301C087554F
:1006E0006A3310F4605301C067556F708295807F44
:1006F000682B862F99270895FC0104C05D9BFECFCF
:1007000031968CB980818823C9F70895982F9295E6
:100710009F708F709A3020F45D9BFECF905D03C078
:100720005D9BFECF995A9CB98A3020F45D9BFECF29
:10073000805D03C05D9BFECF895A8CB9089587E226
:1007400080939A0485E28093990490E290939B04AD
:1007500010929C0428E030E030939E0420939D0486
:1007600083E28093A60481E28093A5049093A7047A
:100770001092A8043093AA042093A9040895089520
:100780006091B20481E20E941007089568E08BE254
:100790000E94100761E188E20E94100768E08FE282
:1007A0000E94100761E18CE20E94100761E08FE275
:1007B0000E9410071092E1011092E00165E083E2CF
:1007C0000E94100708950F931F938C0160E480E24C
:1007D0000E941007F8016281605884E00E941007AF
:1007E000F80182818093B1041F910F9108950F93B6
:1007F0001F93CF93DF93EC012885398512161306DA
:10080000DCF58E819F81821793071CF568E083E2F7
:100810000E94100700E010E00FC08A859B85E80F5A
:10082000F91F608181E20E9410078E819F810196ED
:100830009F838E830F5F1F4FEE81FF81888599858F
:10084000083011051CF4E817F9073CF3E817F9071D
:1008500024F061E087E20E9410078B81813031F43F
:1008600065E089810E9410071B8206C061E08981D2
:100870000E94100781E08B83DF91CF911F910F9130
:100880000895CF93DF93CDB7DEB724970FB6F894D2
:10089000DEBF0FBECDBFDC01FC012281338110928F
:1008A000AC041092AB0481E08093A804832F9927B5
:1008B0008230D9F0833069F1813009F057C08091DE
:1008C000850499279093AE048093AD0485E894E065
:1008D0009093B0048093AF04868197818034910512
:1008E00009F044C088E090E029C0FD01868197812D
:1008F0009093AE048093AD04E22FFF27EE0FFF1F0D
:100900008091970490919804E80FF91F808191815C
:1009100029C02223C1F0E22FFF27EE0FFF1F809195
:10092000F0019091F101E80FF91F0190F081E02DA5
:10093000F093B004E093AF04808199279093AE04C4
:100940008093AD0413C094E0998383E08A8389E0A7
:100950008B839C8384E090E09093AE048093AD04FD
:10096000CE0101969093B0048093AF0485EA94E0A1
:100970000E94F70324960FB6F894DEBF0FBECDBFDA
:10098000DF91CF910895CF93DF9382E20E94E70633
:10099000C82FDD27C5FF1AC068E083E20E94100758
:1009A000C6FF10C02091AB043091AC048091AD041F
:1009B0009091AE04281739072CF485EA94E00E9440
:1009C000F70304C061E087E20E941007DF91CF9136
:1009D00008951F93CF93DF9388E00E94E706182FB6
:1009E000C82FDD27C6FF18C060E085E00E94100711
:1009F00060E884E00E94100760E080E20E94100737
:100A000068E083E20E94100761E087E20E9410071D
:100A100062E085E00E941007C4FF04C060EC89E03A
:100A20000E94100717FF04C060ED89E00E941007C4
:100A3000DF91CF911F9108958AE00E94E7069927E0
:100A400080FF03C00E94C304089581FF0DC08AE2A5
:100A50000E94E70680917204813061F4E091750490
:100A6000F09176040995089582E30E94E7068AE3EF
:100A70000E94E70608958EE00E94E70668E08FE294
:100A80000E94100761E08FE20E9410072091AD04E0
:100A90003091AE048091A9049091AA048217930723
:100AA0005CF468E083E20E94100761E087E20E9444
:100AB000100781E08093A8040895AF92BF92CF926F
:100AC000DF92EF92FF920F931F93CF93DF93CDB7F7
:100AD000DEB728970FB6F894DEBF0FBECDBF86E213
:100AE0000E94E70686FF7EC08E010F5F1F4F5801F0
:100AF00069E0C62ED12CCC0EDD1E809199040E9497
:100B0000E706F80181938F017501EC15FD05A9F742
:100B100068E087E20E94100768E083E20E94100705
:100B200080E20E94E7068F77682F80E20E9410071C
:100B300089819927807690708032910509F440C0B0
:100B400080349105D1F1892BF1F5F5018181863051
:100B5000D9F0873048F48130F1F18130C8F083302A
:100B6000D1F1853081F521C0893019F18A3018F42E
:100B7000883049F505C08A3071F18B3021F520C0ED
:100B8000C5010E94C00327C0C5010E94410423C0C3
:100B900068E083E20E94100761E081E20E94100792
:100BA00060E081E20E9410070BC0C5010E94E303D0
:100BB00012C0C5010E94C6030EC0C5010E94BF0637
:100BC00065E083E206C080E20E94E7068058682F55
:100BD00080E20E941007F70180818823D1F465E04C
:100BE00083E215C02091AD043091AE048091A90438
:100BF0009091AA048217930764F41092AE041092A5
:100C0000AD0468E083E20E94100761E087E20E9481
:100C1000100728960FB6F894DEBF0FBECDBFDF9148
:100C2000CF911F910F91FF90EF90DF90CF90BF90E9
:100C3000AF900895CF92DF92EF92FF920F931F93A0
:100C4000CF93DF93CDB7DEB7C054D0400FB6F89442
:100C5000DEBF0FBECDBF8CE00E94E706992780FF64
:100C600003C00E945D057BC081FF2AC08EE20E9406
:100C7000E7068DE20E94E70689838E010F5F1F4F12
:100C80006801FFE3EF2EF12CE00EF11E0F5F1F4F06
:100C90000E94D306F80180830E151F05B9F78091D5
:100CA0005401813031F4E0915701F0915801C601AF
:100CB000099568E08FE20E94100761E08FE22BC087
:100CC00082FF2CC086E30E94E70685E30E94E706C8
:100CD00089838E010F5F1F4F6801EFE3EE2EF12C29
:100CE000E00EF11E0F5F1F4F0E94D306F8018083B4
:100CF0000E151F05B9F780915501813031F4E0914F
:100D00005901F0915A01C601099568E087E30E94F4
:100D1000100761E087E30E94100721C083FF1FC016
:100D20008EE30E94E7068E010F5F1F4F680171E49A
:100D3000E72EF12CEC0EFD1E8DE30E94E706F80174
:100D400081938F01EE15FF05B9F78091560181302F
:100D500031F4E0915701F0915801C6010995C05C4A
:100D6000DF4F0FB6F894DEBF0FBECDBFDF91CF913E
:100D70001F910F91FF90EF90DF90CF90089508950D
:100D8000089581E08ABF80E189BFE4E6F0E08081D8
:100D900087608083E5E6F0E0808183608083A79AA6
:100DA000AF9A7894089585B3805885BBE5E6F0E066
:100DB000808122E0822780830000000089B395B300
:100DC000905895BB908192279083992708959FEF23
:100DD0009ABB8BBB85B3805885BBE5E6F0E080818C
:100DE00095E08927808385B3805885BB80818927DA
:100DF000808300001ABA0E94D306992708958BBBFE
:100E000085B3805885BBE5E6F0E0808191E08927D5
:100E1000808385B3805885BB80818927808308952E
:100E20008BBB8FEF8ABB85B3805885BBE5E6F0E0CE
:100E3000808195E08927808385B3805885BB808138
:100E400089278083862F0E94FF060895089582E1F6
:100E50008093850481E08093860480E191E0909303
:100E60008804809387041092890410928A04109257
:100E70008B0488E080938C0410928E0410928D0471
:100E80001092900410928F04109292041092910488
:100E90001092930410929404109295041092960468
:100EA0001092540110925501109256011092720442
:100EB000109273041092740410927C0410927B04BC
:100EC0001092EF011092EE01089590938E0480939A
:100ED0008D047093900460938F0450939204409318
:100EE0009104089590938E0480938D0408959093B7
:100EF000900480938F0408959093920480939104BA
:100F0000089580938904089580938A0408958093B6
:100F10008B040895CF93DF939C01CB01E0917B0478
:100F2000F0917C0462E070E00E944E190FC0A08135
:100F3000B1818281823039F4ED018D819927821748
:100F4000930709F468870780F085E02D309779F7DB
:100F5000DF91CF910895CF93DF939C01E0917B04C3
:100F6000F0917C0414C0A081B1818281843061F44D
:100F7000848199278217930739F4868199278617E8
:100F8000970711F4ED014B830780F085E02D309732
:100F900051F7DF91CF910895BF92CF92DF92EF92F8
:100FA000FF920F931F93CF93DF936C01162FF42EB4
:100FB000B22EC0917B04D0917C042097A1F489E0EB
:100FC00090E00E945518FC0190937C0480937B0470
:100FD000D182C082138310861782F282B482058385
:100FE000E68215C0EC018F8198850097D9F789E0DA
:100FF00090E00E945518FC0198878F83D182C082AF
:101000001383F282B4820583E68210861782DF9111
:10101000CF911F910F91FF90EF90DF90CF90BF90F5
:101020000895EF92FF921F93CF93DF937C01C091BD
:10103000EE01D091EF01209711F011E012C085E090
:1010400090E00E945518FC019093EF018093EE010F
:10105000F182E08212821482138210E012C01F5FBC
:10106000EC018B819C810097D1F785E090E00E9494
:101070005518FC019C838B83F182E08212831482D9
:101080001382812F9927DF91CF911F91FF90EF90CD
:101090000895EF92FF920F931F93CF93DF93E09108
:1010A000EE01F091EF0180E090E00380F481E02D0B
:1010B00001963097D1F7880F991F0E945518909389
:1010C000F1018093F0010091EE011091EF01E80130
:1010D000E880F9808A81C82FDD27CC0FDD1F809141
:1010E000F0019091F101C80FD91FF7018081992774
:1010F0000E9455189983888320E030E017C0E801EA
:10110000EA81FF27EE0FFF1F8091F0019091F1011E
:10111000E80FF91F0190F081E02DE20FF31FD701D6
:10112000A20FB31F8C9180832F5F3F4FF701808107
:101130009927281739071CF3E8018B819C810097B8
:1011400011F08C01C4CFDF91CF911F910F91FF90CF
:10115000EF9008954F925F926F927F928F929F923D
:10116000AF92BF92CF92DF92EF92FF920F931F93B5
:10117000CF93DF93E0917B04F0917C046624772485
:1011800009C08281823019F40894611C711C0780A7
:10119000F085E02D3097A9F74301880C991CC40114
:1011A0000E9455189093980480939704E1E0EE2EE6
:1011B000F12CAA24BB2455C0E0917B04F0917C045F
:1011C00079E0C72ED12C15C0A081B18184819927E7
:1011D0008E159F0519F48381C80ED11CED018D81F8
:1011E0008E1521F48281823009F45D010780F0853B
:1011F000E02D309749F70091970410919804025020
:101200001040080D191DC6010E945518F801918360
:10121000808320E030E0E0919704F0919804E80D9D
:10122000F91D32970190F081E02DE20FF31FD501F7
:10123000A20FB31F8C9180832F5F3F4F2930310560
:1012400051F7E0919704F0919804E80DF91D329759
:101250000190F081E02D8C2D875F82830894E11C42
:10126000F11C6E147F040CF0A7CF61E0C62ED12CC8
:1012700059E0A52EB12C4424552442E0842E912C13
:10128000A1C0A0917B04B0917C0412C0ED91FC91AF
:1012900011978181823049F4858199278C159D05AC
:1012A00021F48481482E552405C0ED01AF81B88515
:1012B000109761F731E0E32EF12C79C060917B0447
:1012C00070917C046DC0FB01C081D1818981843023
:1012D00009F063C0868199278E159F0509F05DC0CE
:1012E000848199278C159D0509F057C0950140E030
:1012F00050E0E0919704F0919804E80DF91D3297C1
:101300000190F081E02DE20FF31FDE01A40FB51F65
:101310008C9180832F5F3F4F4F5F5F4F4930510566
:1013200041F789E090E0A80EB91EC0917B04D091EE
:101330007C0431C08A81853059F58C8199278C15C0
:101340009D0531F58D8199278E159F0509F5088139
:101350001981950140E050E0E0919704F0919804E4
:10136000E80DF91D32970190F081E02DE20FF31F97
:10137000D801A40FB51F8C9180832F5F3F4F4F5F23
:101380005F4F4730510541F7E7E0F0E0AE0EBF1E7A
:101390000F80D885C02D209769F6EB016F81788585
:1013A0006115710509F08FCF0894E11CF11C4E14F2
:1013B0005F040CF083CF0894C11CD11CE2E0F0E084
:1013C0008E0E9F1E6C147D040CF05BCFDF91CF91CD
:1013D0001F910F91FF90EF90DF90CF90BF90AF9053
:1013E0009F908F907F906F905F904F9008956F9235
:1013F0007F928F929F92AF92BF92CF92DF92EF92A5
:10140000FF920F93CF93DF935C013B014901E09181
:101410007B04F0917C0416C0A081B181848199275E
:10142000A816B90661F4868199278615970539F4BF
:101430008281843021F4ED018C818F5F8C83078061
:10144000F085E02D309741F787E090E00E94551835
:10145000FC0187E0808385E0818382820383F582BB
:10146000E482C682EE24062D2A2D45E067E0CF01F6
:101470000E94CC07DF91CF910F91FF90EF90DF900A
:10148000CF90BF90AF909F908F907F906F90089576
:10149000AF92BF92CF92DF92EF92FF920F93FC0137
:1014A000A114B10401F14230510571F043305105EE
:1014B00099F041305105B9F481E080937204B09203
:1014C0007604A09275040FC081E080937304B092FB
:1014D0007804A092770407C081E080937404B092EE
:1014E0007A04A092790420583F4FCF010E94F70957
:1014F0000F91FF90EF90DF90CF90BF90AF90089545
:10150000AF92BF92CF92DF92EF92FF920F93FC01C6
:101510004230510571F04330510599F04130510589
:10152000B9F481E080935401B0925801A092570120
:101530000FC081E080935501B0925A01A0925901E9
:1015400007C081E080935601B0925C01A0925B01DC
:10155000CF010E94F7090F91FF90EF90DF90CF909D
:10156000BF90AF900895CF92DF92EF920F931F93A9
:10157000CF93DF936C018B01A0917B04B0917C042D
:10158000C0E0D0E014C02D913C911197F901858104
:101590008C1551F4FD018281823031F4F90184818E
:1015A0008F5F8483C82FDD27FD01A781B085109749
:1015B00051F789E090E00E945518FC0189E0808392
:1015C00084E081830283138214821582168217823B
:1015D0001086EC2E00E02C2D44E069E0CF010E9443
:1015E000CC07CE01DF91CF911F910F91EF90DF904B
:1015F000CF900895BF92CF92DF92EF92FF920F9318
:101600001F93CF93DF936C017B01142FB22EA09117
:101610007B04B0917C04C0E0D0E014C02D913C91DB
:101620001197F90185818C1551F4FD018281823079
:1016300031F4F90184818F5F8483C82FDD27FD0198
:10164000A781B085109751F789E090E00E94551866
:10165000FC0189E0808384E08183E282138214822A
:101660001583B68207831086EC2E00E02C2D44E013
:1016700069E0CF010E94CC07CE01DF91CF911F918D
:101680000F91FF90EF90DF90CF90BF900895EF9271
:101690000F931F93109196041F5F1093960489E097
:1016A00090E00E945518FC0189E0808389E090E079
:1016B0009383828382E0818314821583168280EA79
:1016C00087838AE18087EE2400E020E042E069E041
:1016D000CF010E94CC07812F99271F910F91EF9086
:1016E0000895CF93DF93EC01FC0101900020E9F70E
:1016F000E81BF90BCF01880F991F0E9455189C0118
:10170000FE0101900020E9F7EC1BFD0BEE0FFF1F1F
:10171000DC01EC9383E0F901818340E050E009C0F3
:10172000FE01E40FF51F80818C93FD0111824F5F54
:101730005F4F1296FE0101900020E9F73197EC1BF4
:10174000FD0B4E175F0760F3C9010E94110899272E
:10175000DF91CF910895EF92FF920F931F93CF9354
:10176000DF938C017B01CA010E94710B9C01E09107
:101770007B04F0917C0414C0A081B181828184300B
:1017800061F4848199278017910739F4868199271C
:101790008E159F0511F4ED0128870780F085E02D57
:1017A000309751F7DF91CF911F910F91FF90EF90FC
:1017B00008950F931F93CF93DF938C01CB010E9469
:1017C000710B9C01E0917B04F0917C040FC0A0811F
:1017D000B1818281823039F4ED018D8199278017A2
:1017E000910709F42E830780F085E02D309779F773
:1017F000DF91CF911F910F9108950E94710B1816E0
:10180000190614F48093950408950E94710B18161C
:10181000190614F48093940408950E94710B18160D
:10182000190614F48093930408951F9386E00E9490
:10183000E706992786FF03C00E941A060EC082FFA2
:1018400003C00E941C0509C081FF03C00E94E90477
:1018500004C084FF02C00E943B0587E00E94E706A7
:10186000182F60E087E00E941007612F87E00E9438
:1018700010071F9108950E94AA080E9449080E941B
:101880009F0361E080E00E94100780E00E94E7066D
:1018900080FDFBCF62E081E00E94100760E884E0F9
:1018A0000E94100760E480E20E94100768E083E273
:1018B0000E94100769E087E20E9410076FE08DE048
:1018C0000E9410076FE08BE00E94100768ED89E02E
:1018D0000E94100763E38FE00E94100766ED87E027
:1018E0000E94100762E085E00E9410076CEC80E027
:1018F0000E94100708958EEC80935D0181E087BF00
:1019000080915D0182BF83E083BF089508950895AB
:1019100083E08093320381E0809333038BE08093F4
:1019200034039FE69093350383E68093360384E780
:10193000809337039093380380E78093390385E7DA
:1019400080933A0383E780933B038FE580933C03C6
:1019500080E380933D0381E380933E0310923F0335
:101960008EE090E00E946C010895FC01808183303C
:1019700011F40E94880C0895CF93DF93C1E0D0E06A
:10198000CE010E94D20D2196C431D105C9F7CAE11A
:10199000D0E0CE010E94D20D2196CD32D105C9F7FB
:1019A000DF91CF910895CF93DF93DC01EC01EA81C1
:1019B000FB8121918E81815019F48981E81BF10905
:1019C000ED01FB83EA838E839FB7F8948C9181505D
:1019D0008C939FBF822F9927DF91CF910895FC01AF
:1019E0001082758364837383628341834783468354
:1019F0000895CF93DF93DC019C91ED0189819817C5
:101A000018F080E090E016C0ED01EC81FD8161935B
:101A10008F81815019F48981E81BF109ED018F83D1
:101A2000FD83EC839FB7F8948C918F5F8C939FBF5D
:101A300081E090E0DF91CF910895FC0180818823BF
:101A4000E9F3CF010E94D30C99270895FC0180810E
:101A5000882319F48FEF9FEF0895CF010E94D30CD4
:101A6000992708950895CF93DF93CDB7DEB72297D6
:101A70000FB6F894DEBF0FBECDBF9C010197439710
:101A800028F0C9014A97439708F07DC0F901EE0F8D
:101A9000FF1FE35AFE4F82E090E092838183F901B9
:101AA0003197EC32F10508F06EC0EA5BFF4FEE0FA4
:101AB000FF1F0590F491E02D0994159A5BC0169ACA
:101AC0005DC0179A57C0B89A59C0B99A53C0BA9A0C
:101AD00055C0BB9A4FC0BC9A51C0BD9A4BC0BE9A6C
:101AE0004DC0BF9A47C0889A49C0899A43C08A9A14
:101AF00045C08B9A3FC08C9A41C08D9A3BC08E9A4C
:101B00003DC08F9A37C0A09A39C0A19A33C0A29A1B
:101B100035C0A39A2FC0A49A31C0A59A2BC0A69A0B
:101B20002DC080916100806807C080916100806451
:101B300019C0809161008062809361001BC0809118
:101B4000610080610FC0809161008860F5CF809155
:101B50006100846007C0809161008260EDCF809158
:101B6000610081608093610009C0109A03C0119ADE
:101B700005C0129A81E090E008C0139AE1E0F0E01D
:101B8000FA83E98304C084E090E09A8389838981A1
:101B90009A8122960FB6F894DEBF0FBECDBFDF91BB
:101BA000CF9108959C010197439738F0C9014A9756
:101BB000439718F084E090E00895C9010E94330D26
:101BC00081E090E00895CF93DF93CDB7DEB7229701
:101BD0000FB6F894DEBF0FBECDBF9C0101974397AF
:101BE00028F0C9014A97439708F07DC0F901EE0F2C
:101BF000FF1FE35AFE4F81E090E092838183F90159
:101C00003197EC32F10508F06EC0EE58FF4FEE0F41
:101C1000FF1F0590F491E02D099415985BC016986C
:101C20005DC0179857C0B89859C0B99853C0BA98B2
:101C300055C0BB984FC0BC9851C0BD984BC0BE9812
:101C40004DC0BF9847C0889849C0899843C08A98BA
:101C500045C08B983FC08C9841C08D983BC08E98F2
:101C60003DC08F9837C0A09839C0A19833C0A298C2
:101C700035C0A3982FC0A49831C0A5982BC0A698B2
:101C80002DC0809161008F7707C0809161008F7BAC
:101C900019C0809161008F7D809361001BC080918D
:101CA00061008F7E0FC080916100877FF5CF8091AA
:101CB00061008B7F07C0809161008D7FEDCF8091A7
:101CC00061008E7F8093610009C0109803C0119855
:101CD00005C0129881E090E008C01398E1E0F0E0C0
:101CE000FA83E98304C084E090E09A838983898140
:101CF0009A8122960FB6F894DEBF0FBECDBFDF915A
:101D0000CF91089580E090E0089580E090E00895FC
:101D100080E090E008950895089508950895089545
:101D2000089508959C01FC01EE0FFF1FE35AFE4F3A
:101D300081819281029719F085E090E00895F90180
:101D40003197EC32F10540F4E256FF4FEE0FFF1FE2
:101D50000590F491E02D099484E090E00895672BBC
:101D600011F01D9AFFC01D98FDC0672B11F01E9A3F
:101D7000F9C01E98F7C0672B11F01F9AF3C01F9887
:101D8000F1C0672B11F0C09AEDC0C098EBC0672B73
:101D900011F0C19AE7C0C198E5C0672B11F0C29A53
:101DA000E1C0C298DFC0672B11F0C39ADBC0C398B3
:101DB000D9C0672B11F0C49AD5C0C498D3C0672B83
:101DC00011F0C59ACFC0C598CDC0672B11F0C69A47
:101DD000C9C0C698C7C0672B11F0C79AC3C0C798BF
:101DE000C1C0672B11F0909ABDC09098BBC0672B03
:101DF00011F0919AB7C09198B5C0672B11F0929AE3
:101E0000B1C09298AFC0672B11F0939AABC0939872
:101E1000A9C0672B11F0949AA5C09498A3C0672B12
:101E200011F0959A9FC095989DC0672B11F0969AD6
:101E300099C0969897C0672B11F0979A93C097987E
:101E400091C0672B11F0A89A8DC0A8988BC0672B02
:101E500011F0A99A87C0A99885C0672B11F0AA9A9A
:101E600081C0AA987FC0672B11F0AB9A7BC0AB985A
:101E700079C0672B11F0AC9A75C0AC9873C0672B12
:101E800011F0AD9A6FC0AD986DC0672B11F0AE9A8E
:101E900069C0AE9867C0672B21F0809162008068AE
:101EA0000DC0809162008F7709C0672B21F080916F
:101EB0006200806403C0809162008F7B8093620027
:101EC00051C0672B21F0809162008062F7CF809132
:101ED00062008F7DF3CF672B21F0809162008061DB
:101EE000EDCF809162008F7EE9CF672B21F080914A
:101EF00062008860E3CF80916200877FDFCF672B2D
:101F000021F0809162008460D9CF809162008B7F44
:101F1000D5CF672B21F0809162008260CFCF809176
:101F200062008D7FCBCF672B21F0809162008160B2
:101F3000C5CF809162008E7FC1CF672B11F0189AB8
:101F400011C018980FC0672B11F0199A0BC019987F
:101F500009C0672B11F01A9A05C01A9803C0672BA5
:101F600021F01B9A81E090E008951B9881E090E0B9
:101F70000895CF93DF93EC010197439738F0CE019A
:101F80004A97439718F084E090E013C0FE01EE0FEB
:101F9000FF1FE35AFE4F83E090E092838183CE01DE
:101FA0000E94330D61E070E0CE010E94920E81E04C
:101FB00090E0DF91CF91089508959C01DB01119687
:101FC0001C921E92FC01EE0FFF1FE35AFE4F81810F
:101FD00092818130910519F085E090E008952130DB
:101FE000310531F4859B28C011963C932E9324C073
:101FF0002230310531F4869B2AC011969C938E9332
:1020000026C02330310531F40F9B2CC011969C93D0
:102010008E9328C02430310531F4B09B2EC0119628
:102020009C938E932AC02530310531F4B19B30C08A
:1020300011969C938E932CC02630310541F4B29BAF
:1020400032C081E090E011969C938E932CC0273093
:10205000310541F4B39B32C081E090E011969C932E
:102060008E932CC02830310541F4B49B32C081E0FE
:1020700090E011969C938E932CC02930310541F449
:10208000B59B32C081E090E011969C938E932CC05A
:102090002A30310541F4B69B32C081E090E01196C0
:1020A0009C938E932CC02B30310541F4B79B32C0EA
:1020B00081E090E011969C938E932CC02C303105DA
:1020C00041F4809B32C081E090E011969C938E9306
:1020D0002CC02D30310541F4819B32C081E090E06D
:1020E00011969C938E932CC02E30310541F4829B27
:1020F00032C081E090E011969C938E932CC02F30DB
:10210000310541F4839B32C081E090E011969C93AD
:102110008E932CC02031310541F4849B32C081E084
:1021200090E011969C938E932CC02131310541F49F
:10213000859B32C081E090E011969C938E932CC0D9
:102140002231310541F4869B32C081E090E0119646
:102150009C938E932CC02331310541F4879B32C070
:1021600081E090E011969C938E932CC02A3131052A
:1021700041F4809B32C081E090E011969C938E9355
:102180002CC02B31310541F4999B32C081E090E0A5
:1021900011969C938E932CC02C31310541F49A9B5F
:1021A00032C081E090E011969C938E932CC02D312B
:1021B000310541F49B9B32C081E090E011969C93E5
:1021C0008E932CC02E31310541F49C9B32C081E0AE
:1021D00090E011969C938E932CC02F31310541F4E1
:1021E0009D9B32C081E090E011969C938E932CC011
:1021F0002032310541F49E9B32C081E090E011967F
:102200009C938E932CC02132310541F4079B32C040
:1022100081E090E011969C938E932CC02232310580
:1022200041F4069B32C081E090E011969C938E931E
:102230002CC02332310541F4059B32C081E090E08F
:1022400011969C938E932CC02432310541F4049B4B
:102250002AC081E090E011969C938E9324C0253291
:10226000310541F4039B25C081E090E011969C93D9
:102270008E931FC02632310541F4029B20C081E0BD
:1022800090E011969C938E931AC02732310541F449
:10229000019B1BC081E090E011969C938E9315C02A
:1022A0002832310519F02932310519F4809B17C005
:1022B00011C02A32310519F4099B11C00BC02B3211
:1022C000310519F40A9B0BC005C02C32310539F4D5
:1022D0000B9B05C081E090E08D939C93089581E075
:1022E00090E008950895CF93DF93CDB7DEB722979E
:1022F0000FB6F894DEBF0FBECDBF2BE120933203A3
:10230000BE016F5F7F4F0E94DD0F80933303898191
:102310008093340383E090E00E946C0122960FB614
:10232000F894DEBF0FBECDBFDF91CF9108952AE1B3
:10233000209332030E94920E809333031092340351
:1023400083E090E00E946C01089527E1209332031E
:102350000E94B90F809333031092340383E090E01E
:102360000E946C01089525E1209332030E94E30D41
:10237000809333031092340383E090E00E946C0159
:10238000089526E1209332030E94330D8093330396
:102390001092340383E090E00E946C01089521E1E3
:1023A000209332030E94D20D8093330310923403A2
:1023B00083E090E00E946C010895FC0180818631E9
:1023C000E9F0873138F48531A0F48231C0F58031ED
:1023D00058F10AC08A3118F4883188F514C08A315E
:1023E000B9F08B3109F51BC0828199270E94CF116A
:1023F0000895828199270E94B311089582819927B7
:102400000E94C1110895828199270E94B90F0895F1
:1024100063817727828199270E949711089582818D
:1024200099270E94731108958093320383E080936B
:1024300033031092340383E090E00E946C0108950E
:10244000FC018197089718F084E090E00895EE0F62
:10245000FF1FE35AFE4F84E090E09283818381E086
:1024600090E0089517B88230910541F083309105CE
:1024700049F0019721F082E090E008953E9A81E0D2
:1024800090E0089587B1806C87B981E090E008956D
:1024900093E896B997B1907F982B97B9369A369969
:1024A000FECF84B195B120E030E040E050E0369AB4
:1024B0003699FECF84B195B1480F591F2F5F3F4F1A
:1024C00024303105A1F73798CA01969587959695DE
:1024D00087950895CF93DF939C01EB0119821882B1
:1024E000FC01EE0FFF1FE35AFE4F8181928104979A
:1024F000D1F52432310559F12532310554F4223217
:10250000310559F1233231052CF52132310559F5C8
:1025100027C026323105A9F026323105ACF027322A
:10252000310531F028323105F1F480E090E002C04D
:1025300081E090E00E9448129983888381E090E0D6
:1025400014C082E090E0F6CF83E090E0F3CF84E027
:1025500090E0F0CF85E090E0EDCF86E090E0EACF2C
:1025600087E090E0E7CF85E090E0DF91CF9108959C
:1025700022E2209332030E9432128093330382E0DE
:1025800090E00E946C010895CF93DF93CDB7DEB742
:1025900022970FB6F894DEBF0FBECDBF21E2209385
:1025A0003203BE016F5F7F4F0E946A128093330334
:1025B00029813A81832F992780933403209335030F
:1025C00084E090E00E946C0122960FB6F894DEBF82
:1025D0000FBECDBFDF91CF91089520E2209332034B
:1025E0000E942012809333031092340383E090E022
:1025F0000E946C010895FC018081813249F0823291
:1026000061F0803279F4828199270E94ED12089559
:10261000828199270E94C4120895828199270E947D
:10262000B81208958093320383E0809333031092AD
:10263000340383E090E00E946C0108958091710062
:102640009927887F907008958091740087FFFCCF50
:102650000895E4E7F0E08081846080838BE090E07F
:1026600090937701809376018CE090E090937901CC
:102670008093780181E090E00895E4E7F0E08081C4
:102680008B7F808382E090E0909377018093760146
:10269000909379018093780108958130910511F428
:1026A0008CE00BC08230910511F488E106C00397DD
:1026B00019F082E090E0089588E4809370008091A2
:1026C00071008C7F80937100809171008093710004
:1026D00081E090E008958091710084EA8093740015
:1026E0008091740087FFFCCF81E090E0089584E939
:1026F0008093740081E090E008958093730084E8F3
:10270000809374008091740087FFFCCF80E090E09C
:10271000089584E8809374008091740087FFFCCF53
:10272000809173009927089585E38093320381E0B7
:10273000809333038093340384E880937400809102
:10274000740087FFFCCF809173008093350385E090
:1027500090E00E946C01089540E050E00FC0F90144
:10276000E40FF51F80818093730084E880937400E8
:102770008091740087FFFCCF4F5F5F4F461757076C
:1027800074F384E38093320381E0809333031092E7
:10279000340383E090E00E946C01089587E3809306
:1027A000320384E98093740081E0809333031092B4
:1027B000340383E090E00E946C01089586E38093E7
:1027C00032038091710084EA8093740080917400D8
:1027D00087FFFCCF81E0809333031092340383E0C2
:1027E00090E00E946C01089522E3209332030E943E
:1027F0004D13809333031092340383E090E00E94E2
:102800006C01089581E380933203E4E7F0E0808176
:102810008B7F808382E090E09093770180937601B4
:1028200090937901809378011092330310923403CE
:1028300083E090E00E946C01089580E3809332036E
:10284000E4E7F0E08081846080838BE090E0909307
:102850007701809376018CE090E0909379018093EA
:10286000780181E0809333031092340383E090E099
:102870000E946C010895FC0180818433D9F0853376
:1028800038F4813379F0823381F0803389F507C0E1
:10289000863341F18633D8F0873351F526C00E9444
:1028A0001D1408950E9402140895828199270E94A0
:1028B000F413089542815527618177276450704051
:1028C000838134969F0199270E94AC130895428119
:1028D00055276181772764507040838199270E9432
:1028E000941308950E94DE1308950E94CE13089554
:1028F0008093320383E0809333031092340383E0A8
:1029000090E00E946C01089588B3817F88BBBB98DA
:1029100086E087BB1DB81EB883E58DB988E090E0DE
:1029200090936901809368018AE090E090936B0135
:1029300080936A0189E090E090936D0180936C012F
:1029400081E090E008951DB81EB882E090E0909379
:1029500069018093680190936B0180936A01909361
:102960006D0180936C0181E090E00895089581E00D
:1029700090E00895AC0120E030E009C0FA01E20FD8
:10298000F31F80818FB9779BFECF2F5F3F4F2617B4
:102990003707A4F381E090E00895DC0120E030E007
:1029A00040E050E014C01FB809C04F5F5F4F83E0A4
:1029B000493E58071CF086E090E00895779BF5CFDC
:1029C000FD01E20FF31F8FB180832F5F3F4F26176A
:1029D00037074CF381E090E00895CF93DF93EC014B
:1029E00020E030E0A0E0B0E017C0FE01E20FF31FEE
:1029F00080818FB908C0119683E0A93EB8071CF00A
:102A000086E090E00EC0779BF6CFFB01E20FF31F4C
:102A10008FB180832F5F3F4F2417350734F381E058
:102A200090E0DF91CF9108950F931F938B0123E4E2
:102A300020933203AB0164E373E00E94ED148093B2
:102A4000330310923403C80102960E946C011F9157
:102A50000F9108950F931F938C0184E480933203A8
:102A6000B80184E393E00E94CD1480933303109265
:102A70003403C80102960E946C011F910F910895C2
:102A800023E4209332030E94BA14809333031092FC
:102A9000340383E090E00E946C01089581E4809308
:102AA00032030E94A314809333031092340383E013
:102AB00090E00E946C01089580E4809332030E94AC
:102AC0008414809333031092350383E090E00E94D6
:102AD0006C010895CF93DF93EC0188818334A1F0DA
:102AE000843438F4813469F0823458F58034F1F458
:102AF00005C0843481F08534C9F411C00E945C158E
:102B000020C00E944E151DC069817727CE01029614
:102B10000E94401516C0898199270E942A15698153
:102B20007727CE0102960E9414150BC080933203C2
:102B300083E0809333031092340383E090E00E949B
:102B40006C01DF91CF910895B89AB99ABA9ABB985F
:102B5000BC9ABD9AC498C59882E090E09093850194
:102B600080938401909383018093820190938101EB
:102B70008093800181E090E090937F0180937E01BB
:102B8000089582E090E090936901809368019093AA
:102B90006B0180936A0190936D0180936C0181E0D9
:102BA00090E00895C098C198C29880E29EE4019791
:102BB000F1F7C09A8AE0982F9A95F1F7C29AC19AD4
:102BC0008A95F1F70895282FC19887FD02C0C29811
:102BD00001C0C29A8AE0982F9A95F1F7C19A8A9516
:102BE000F1F7C19826FF02C0C29A01C0C2988AE0DC
:102BF000982F9A95F1F7C19A8A95F1F70895282FA1
:102C0000220F30E0C19827FF02C0C29A01C0C298CB
:102C10008AE0982F9A95F1F7C19A8A95F1F73F5F6C
:102C2000373011F0220FEECF0895282F30E0C198F1
:102C300027FF02C0C29A01C0C2988AE0982F9A95D5
:102C4000F1F7C19A8A95F1F73F5F383011F0220F02
:102C5000EECF0895C198C2988AE0982F9A95F1F71F
:102C6000C19A982F9A95F1F7C198C098982F9A9584
:102C7000F1F7C19A982F9A95F1F7C1988A95F1F7D3
:102C8000C09A80E090E00895C198C098C298C39A15
:102C900008950E94D21580E30E94E31580E60E9409
:102CA000FF1508950E94D21580E00E94E31580E090
:102CB0000E94FF150E94441608950F931F93182F2A
:102CC000062F0E94D21580E40E94E315812F0E94F6
:102CD000FF15802F0E94151681E090E01F910F9143
:102CE00008951F93182F0E94D21580EC0E94E315BF
:102CF000812F0E94FF150E942A1699271F9108957F
:102D0000C1988AE08A95F1F7C29830E090E0990F77
:102D1000C19A2AE0822F8A95F1F7C198B3999F5FF3
:102D2000822F8A95F1F73F5F383089F7C098C19AB2
:102D3000822F8A95F1F7C09AC1982A95F1F7892FC9
:102D4000992708951F93182F0E94D21580E80E949A
:102D5000E315812F0E94FF150E94801699271F916D
:102D60000895DF92EF92FF920F931F93CF93DF931B
:102D7000D82E7B018A01C0E0D0E009C08D2D8C0FD8
:102D80000E94A216F801EC0FFD1F80832196CE153C
:102D9000DF05A1F781E090E0DF91CF911F910F91C6
:102DA000FF90EF90DF9008950F931F93082F162F39
:102DB0000E944916612F802F0E945D1681E090E0ED
:102DC0001F910F910895DF92EF92FF920F931F933F
:102DD000CF93DF93D82E7B018A01C0E0D0E009C0F9
:102DE000F801EC0FFD1F60818D2D8C0F0E94D41611
:102DF0002196CE15DF05A1F781E090E0DF91CF911C
:102E00001F910F91FF90EF90DF90089594E09093C1
:102E100032030E94E316809333031092340383E05D
:102E200090E00E946C0108950F931F938B0193E033
:102E30009093320344E353E00E94B116809333032E
:102E4000C80102960E946C011F910F91089582E0C3
:102E50008093320382E090E090936901809368014F
:102E600090936B0180936A0190936D0180936C0144
:102E700081E0809333031092340383E090E00E945A
:102E80006C01089581E0809332030E94A415809321
:102E900033031092340383E090E00E946C010895A4
:102EA000FC018381823069F0833018F48130F1F4C1
:102EB00005C0833049F08430C9F40FC00E94421726
:102EC00008950E9427170895AF014A5F5F4F6581FB
:102ED000772784810E9414170895AF014A5F5F4FDE
:102EE0006581772784810E940617089580818093E9
:102EF000320383E0809333031092340383E090E045
:102F00000E946C0108951F920F920FB60F92112428
:102F10008F939F938091B3049091B4049BBD8ABD1D
:102F20009F918F910F900FBE0F901F901895FC01ED
:102F30000897029718F084E090E00895EE0FFF1FC5
:102F4000E35AFE4F8DE090E09283818381E090E030
:102F500008959C01FC01EE0FFF1FE35AFE4F818193
:102F600092810D97F1F428303105F1F029303105C7
:102F7000C1F48091B3049091B404892B31F480E8BA
:102F800090E09093B4048093B3046130710561F4D0
:102F90008FB5816A8FBD8EB581608EBD81E090E076
:102FA000089585E090E0089581E090E008959C0107
:102FB000FC01EE0FFF1FE35AFE4F818192810D97B6
:102FC00059F42830310529F02930310529F47BBD29
:102FD0006ABD81E090E0089585E090E008959C014D
:102FE00082E580933203F901EE0FFF1FE35AFE4F93
:102FF000818192810D9759F42830310529F02930CB
:10300000310529F47BBD6ABD81E090E002C085E016
:1030100090E0809333031092340383E090E00E94A9
:103020006C01089521E5209332030E94A917809333
:1030300033031092340383E090E00E946C01089502
:1030400020E5209332030E94971780933303109258
:10305000340383E090E00E946C010895FC018081BC
:10306000813549F0823571F0803599F48281992754
:103070000E942018089563817727828199270E94F2
:103080001218089563817727828199270E94EF178C
:1030900008958093320383E08093330310923403C6
:1030A00083E090E00E946C010895CF93DF93AC0120
:1030B000029710F442E050E0A091B704B091B80438
:1030C000FD01C0E0D0E020E030E020C080819181AF
:1030D0008417950769F482819381209719F09B8367
:1030E0008A8304C09093B8048093B704CF0132C0A0
:1030F0004817590738F42115310519F0821793073D
:1031000008F49C01EF010280F381E02D3097F1F685
:103110002115310589F1C901841B950B049708F429
:10312000A901E0E0F0E026C08D919C9111978217F3
:103130009307E9F44817590779F4ED018A819B81D7
:10314000309719F09383828304C09093B8048093DE
:10315000B704CD01029649C0841B950BFD01E80F11
:10316000F91F4193519302978D939C933AC0FD01AF
:10317000A281B3811097C1F68091B5049091B604F5
:10318000892B41F480915001909151019093B604A4
:103190008093B504209152013091530121153105DE
:1031A00041F42DB73EB780914E0190914F01281BFD
:1031B000390BE091B504F091B6042E1B3F0B241798
:1031C000350788F0CA0102962817390760F0CF0149
:1031D000840F951F02969093B6048093B504419393
:1031E0005193CF0102C080E090E0DF91CF9108952C
:1031F000CF93DF93009709F44EC0EC0122971B8216
:103200001A82A091B704B091B804109711F140E070
:1032100050E001C0DC01AC17BD0700F1BB83AA83FD
:10322000FE0121913191E20FF31FEA17FB0771F4C0
:103230002E5F3F4F8D919C911197820F931F998321
:103240008883FD01828193819B838A834115510587
:1032500059F4D093B804C093B7041DC0FD01828116
:103260009381AD010097B1F6FA01D383C283219116
:103270003191E20FF31FEC17FD0769F42E5F3F4F0A
:1032800088819981820F931FFA01918380838A81BB
:103290009B8193838283DF91CF91089597FB092EC1
:1032A00007260AD077FD04D027D006D000201AF4D4
:1032B000709561957F4F0895F6F7909581959F4F92
:1032C000089597FB092E05260ED057FD04D028D06F
:1032D0000AD0001C38F450954095309521953F4F09
:1032E0004F4F5F4F0895F6F79095809570956195D3
:1032F0007F4F8F4F9F4F0895AA1BBB1B51E107C003
:10330000AA1FBB1FA617B70710F0A61BB70B881F75
:10331000991F5A95A9F780959095BC01CD01089504
:10332000A1E21A2EAA1BBB1BFD010DC0AA1FBB1FC9
:10333000EE1FFF1FA217B307E407F50720F0A21B3B
:10334000B30BE40BF50B661F771F881F991F1A94A8
:1033500069F760957095809590959B01AC01BD01D2
:04336000CF010895FC
:10336400456D62656464656450726F6A6563747305
:10337400004F63746F70757355534220496E7465C2
:10338400726661636520436F6E7665727465722040
:10339400616E6420492F4F20457874656E73696FA0
:1033A4006E003230303831313038000904002000EA
:0433B400B904000058
:00000001FF
